:020000020000FC
:100000005CCEC1C10000000020C0000093C0000011
:1000100000009DC000000000000000000203040674
:10002000080C10182030406080000406080C1018DE
:100030002030406080A0C00000070F1F3F000D0D62
:100040000403060D0503030202004FB662FD0EC055
:10005000552009F00994C52DC095089483FDC795D6
:10006000C4BDC093A10064604FBE1895C0916400E8
:10007000089483FDC795C4BDC093A1006B7FC09158
:100080006400CF3F09F41FC070FF02C082FD05C0AD
:100090004FBEC098AC9895981895C098AC98959814
:1000A00075FD0DC065FD0BC0C9E0CA95F1F7C091A3
:1000B000B300C0FDAB9AC1FDAD9AC2FD949A2092E7
:1000C000A1004FBE189524BCCC27C064C8BF646093
:1000D000F6CFC1CF70FFBFCF65FDBDCFC09ABBCFFC
:1000E00070FFB9CF65FDB7CFAC9AB5CF70FFB3CF76
:1000F00065FDB1CF959AAFCFAB9870FFACCF65FDE2
:10010000AACFC7E0CA95F1F7C09AA5CFAD9870FF06
:10011000A2CF65FDA0CFC7E0CA95F1F7AC9A9BCFFF
:10012000949870FF98CF65FD96CFC7E0CA95F1F718
:10013000959A91CF4FB6C9B7CF7EC9BF6E7FCCB568
:10014000CE0DDDB5DF1DDBBDCABD4FBE18953FB678
:100150008F7EABB7A074A2118061A0E0ABBFA9B73E
:10016000AE7FA9BF7894A0916800AA2341F085FDD5
:100170002AC0A0916800AA95A093680024C040E01E
:1001800050E085FD14C0A0B396FDA095A2FD4FEFF1
:10019000A3E096FDA2E0A5BFAA27A064AABF8D7F19
:1001A000A0B396FDA095A2FD5FEF451741F7A0E42F
:1001B00061FDA093680085FD03C0A0E4A0936800E2
:1001C00040939700816085FD0EC0A0916900AA232D
:1001D00031F0A0916900AA95A093690004C08061E4
:1001E000AA27A064AABF80FF0AC0A09197004A2F47
:1001F00061FF8E7F85FD01C000C04093610040918A
:10020000B600443009F004C0A0916100A0936300DF
:10021000A52DA03408F06860A0916000A395A0937C
:10022000600051F0F894A9B7A160A9BF84FF02C093
:10023000A0E4ABBF3FBE1895A0917400A395A09316
:10024000740042E050916800552329F085FF03C0F7
:100250005A9550936800A0919700A13018F0209211
:100260009A000DC020929B002092A500A0919A00B8
:10027000AF5FA0939A0018F0AFEFA0939A00B090F0
:1002800061005091B600523049F466FF91F0A2E34C
:10029000BA1678F0A0918700A0936100533049F41A
:1002A00066FF39F0A2E3BA1620F0A091C200A09335
:1002B0006100509162005B1521F010F05A9501C069
:1002C0005395509362004A95D1F65091A5005395ED
:1002D00009F45A955093A500A091A600AA95A09361
:1002E000A60009F046C0A1E0A093A60045E0A091B9
:1002F000A7005A17F0F1A091A8005A1728F441E07E
:10030000A3E0A093A60007C0A091A9005A1718F473
:1003100041E04093A600D0909D00C0906300DC14A3
:10032000A8F0A091B600A430D9F066FD0FC0C0922D
:100330009D00539511F0A091A700A093A500A1E006
:10034000A093A600ACE3A093620013C0A0919D000F
:10035000A40F20F45FEF50939D0002C0A0939D0076
:10036000A0919D00AF3F29F4AFEFA0939B00A09315
:10037000A500F894A9B7A160A9BF84FF02C0A0E4BA
:10038000ABBF3FBE18953FB64CB55DB58F7EABB7E2
:10039000A074A2118061A0E0ABBFA9B7AE7FA9BFD6
:1003A000789481FD23C0A2E096FDA3E0A5BF826002
:1003B000A0B396FDA095A2FF05C0409365005093A1
:1003C00066001CC1A3E096FDA2E0A5BFAA27A06419
:1003D000AABF8D7F85FF01C004C140E0A0B396FD98
:1003E000A095A2FDFEC040939700EDC0A3E096FD4E
:1003F000A2E0A5BF8D7F61FF71C0A2E096FDA3E0E2
:10040000A5BFAA27A064AABF826040939200509320
:100410009300A09090004A19B09091005B09BB2412
:10042000A22C4C38520518F42092960049C0A09195
:10043000D600AA2359F1483C520528F4A0E1BA2E6F
:10044000AAE0AA2E23C04836A1E05A0728F4A8E063
:10045000BA2EAFE0AA2E1AC0403DA2E05A0728F4F7
:10046000A4E0BA2EAEE1AA2E11C0403AA5E05A0788
:1004700028F4A2E0BA2EACE3AA2E08C04839A8E0BE
:100480005A0720F4A1E0BA2EA8E7AA2EC42EA09104
:100490009400CA1AD52EA0919500DA0ADD202AF41C
:1004A000AFEFC094D094CA1ADA0A20929600A8E05E
:1004B000A210A0E0CA14DA0618F4A1E0A0939600F6
:1004C0004093940050939500409192005091930076
:1004D000409390005093910002E075C0A091650098
:1004E0004A1BA09166005A0B94FD60C093FD5EC04C
:1004F00092FD5AC086FF03C0D52EC42E0CC056955F
:10050000479591FD51C05695479590FD4DC0D52E0C
:10051000C42ED694C79461FD19C0AC2DAC51AD2D3D
:10052000A24008F005C0DD2089F4AC2DA85C70F471
:10053000A0916700A395AA2311F0A0936700AA30A9
:1005400008F44FC02092970081604BC0A0916700D3
:10055000AA2319F0AA95A0936700A22C5091BC0081
:1005600097FD02C0A090CA00AAEFAA0EA22DA21D5C
:10057000CA18DA0A4FB74170442319F040E050E03E
:1005800015C0AFEFCA16D20418F04FEF50E00EC0FE
:10059000A091AE00CA9E412D000C441F50E008F00F
:1005A00012C04FEF50E00FC05695479594FF07C01B
:1005B000552309F04FEFA42FA6954A0F521D4F3F28
:1005C000520508F04FEF40939700816061FF09C02A
:1005D000AFE1A095A923AB299A2F8F7DBB2009F409
:1005E0008062A0E4A093680085FF03C0AAE0A09306
:1005F000680061FD03C085FD01C08F7E85FD03C0DD
:10060000A0E2A0936900F894A9B7A160A9BF84FFF4
:1006100002C0A0E4ABBF3FBE189511E00AC013E0D2
:1006200008C01AE006C01EE104C014E602C018ECBF
:1006300000C005E1BB27BA95F1F70A95D9F71A95DD
:10064000C1F708952AE338E709C020E33CE806C073
:100650002AE234EB03C025E238EC00C012E095FD3D
:100660009F7D95FF9062BB27AD98BA95F1F7AC9A44
:10067000BA95F1F7AC98BA95F1F7AD9ABA95F1F74A
:10068000C09AB091AF00BA95F1F7C098B7E8BA95A3
:10069000F1F71A9521F7022FB22FBA95F1F70A95C3
:1006A000D9F73A95D9F6AD980895221B39E0001F85
:1006B0003A9509F40895221F211B18F4210F8894FC
:1006C000F6CF0894F4CF622C722CB0E08894B395E6
:1006D000221F331FE0F7379527958894912E802E9F
:1006E000020B130B10F4192D082D10F4889401C07F
:1006F0000894661C771CBA9571F7172D062D08957E
:10070000322D11232AF43A9500951095031B130BF3
:10071000F894029F712C002D129F912C802C7894BC
:10072000780C172D921C292DB4E06B2E2695179569
:1007300007956A94D9F7332321F000951095031B90
:10074000130B08950091B600043009F474C0B09101
:100750009700B95198F0B72FB67081F466FD2BC0A1
:1007600005E09090C800B92DBA9521F00AE0BA953D
:1007700009F002E1B0917B00B01BE0F066FF0AC017
:10078000B0919F00B0939D00BFEFB093A500B1E082
:10079000B093A600B0916100B093630020927F00F7
:1007A000209280002092810020928200209283007B
:1007B0006F7B41C060649090C800B92DBA9579F400
:1007C000B0916200B095BB1FBB1F1B2FB7950B2FBD
:1007D000B12FB170B3951B2FB02FBE7F25C0B92D9F
:1007E000BA95BA9581F4B0916200B095BB1FBB1F5A
:1007F000BB1F1B2FB7950B2FB12FB370B3951B2FBA
:10080000B02FBC7F14C0B0916200B095BB1FBB1F5E
:10081000BB1FBB1F1B2FB7950B2FB12FB770B39505
:10082000B3951B2FB02FB87FB0540B2F1209009334
:100830007F0010938000089510917B001695009121
:100840007A000795B0917F00B01B0B2FB09180000C
:10085000B10B1B2F28F40038BFEF1B0740F009C075
:100860000F37120508F405C00FE710E002C000E8DA
:100870001FEF009384001093850008950091840079
:10088000B09181000B0F10918500B09182001B1F69
:1008900020E03091850033230AF42A95B09183003B
:1008A0002B1F1AF4203F40F00AC02F3008F407C075
:1008B0000FEF1FEF2FE003C000E010E020EF3091BA
:1008C0006300B0919C003B1718F4323030F009C03F
:1008D000B0918500BB235AF004C0B0918500BB23C2
:1008E00032F40093810010938200209383000895D6
:1008F0002091D80000918400000F10918500111FF5
:10090000FFDE11232AF40038BFEF1B0740F009C0B7
:100910000F37120508F405C00FE710E002C000E829
:100920001FEF002352F0B0916200B01B0B2F18F0A4
:10093000013008F00AC001E008C000950F5FB091D7
:1009400062000B0F08F001C00FEF009386000895BE
:100950002091D9000091820010918300D1DE1123F3
:100960002AF40130BFEF1B0740F009C00F3F12050A
:1009700008F405C00FEF10E002C001E01FEF1123E3
:1009800052F0B0918600B01B0B2F18F0013008F028
:100990000AC001E008C000950F5FB09186000B0F00
:1009A00008F001C00FEF0093630008950FEF677F19
:1009B00071FD29C072FD09C06860B0917B00BA303A
:1009C00020F0B52DB03408F4677FB091D500BB237B
:1009D000D1F0B0917B00BB23B1F00FEF10917B0001
:1009E00064DEF894B091730072FDB5E00B9F112D99
:1009F000002D7894112309F00FEFB0919F000B1791
:100A000010F400919F0000939E00089500917A00D9
:100A100010917B0000541140B0919E0010F4BA95E3
:100A200001C0B39511F0B0939E000895F3D3B2E0E6
:100A300073FDB1E0B7B9B6B1B068B064B6B9EDDD79
:100A4000B2E073FDB1E0B7B9B6B1B068B064B6B9A1
:100A5000B6B1B6FDFDCF04B115B1B6B1BF77B6B929
:100A60002CD424E72093AA00222309F441C030E0CB
:100A70003093AB00732E7694622E6694620E731ED2
:100A8000262D372D0217130778F08090AA00B4E7BF
:100A9000B80DB093AA008090AB00B0E0B81DB09341
:100AA000AB00260D371DEECF8090AA009090AB00D2
:100AB0001091AB0016950091AA0007951695079521
:100AC00023E0169507952A95E1F72091B7002A951E
:100AD00029F42092AA002092AB000AC02A9521F0A6
:100AE000800E911E2A95E1F78092AA009092AB00A9
:100AF00008952091B700B6B1B6FDFBCF04B115B192
:100B0000B6B1BF77B6B9B091AC00B395B093AC00B5
:100B1000B83060F12092AC00B091D400BB2321F139
:100B2000112329F0B091AD00BF3F61F009C0B09131
:100B3000AD000B1739F020F4BB2321F0BA9502C0A9
:100B4000B395E1F300919C00B093AD00B13A50F43D
:100B500000ECB43938F400E8B73820F400E4BA37D0
:100B600008F400E000939C00777F08952130B1F0F5
:100B70000F3FB3E01B0790F4B4E7BB2379F0B091CB
:100B8000AA000B17B091AB001B0740F4B0919C007A
:100B9000BB2359F0BA95B0939C0007C0B0919C005C
:100BA000BF3F19F0B395B0939C0000919C00B091A9
:100BB0006300B01B10F400916300B0919D000B170F
:100BC00050F000919D00B0919D00BF3F21F0B09189
:100BD0009D00B0939C00502E00936400B091AC0037
:100BE000B73009F47860089502E3F894B091DA0020
:100BF0000B9F012D000C001F7894B0919C000B17E7
:100C000010F000919C000093610000936300502E4F
:100C10000093640000939F00089520927A00B0EF43
:100C2000B0937B000895F8940CB51DB52091740025
:100C30007894309175006090760000937500109361
:100C40007600031B160971FD03C076FD81C02BC021
:100C500070907700209377002709222311F00FEF7F
:100C60001FEF809078009090790030937800609228
:100C700079006918161910937C0000917500109185
:100C800076000819190920917A0030917B00369579
:100C90002795020F131F10F40FEF1FEF00937A0038
:100CA00010937B0029C020917A0030917B0039019C
:100CB000B4E08B2EB2E09B2E343010F08A949A94DC
:100CC000383010F08A949A94769467948A94E1F775
:100CD00026193709992021F0169507959A94E1F77E
:100CE000200F311F20937A0030937B0028F43FEFD0
:100CF00030937A0030937B00323008F4706471FFD7
:100D000002C0B3E00DC0B091C6000091710002387E
:100D100038F0B395003A08F0B395B63008F0B5E076
:100D20009B2EB4E08B2E10917B0000917A0024E082
:100D3000169507952A95E1F70819120928F0B02FA2
:100D4000B250B12FB20910F402E010E0980126C0B1
:100D500020917A0030917B003901769467946694F3
:100D6000669466942619320906950695200F321D61
:100D700020937A0030937B00323008F07F7B04E0D0
:100D8000369527953695279526952695201B10F0A4
:100D9000223008F422E089019090C60060FDFECF69
:100DA000E0908C00F0908D006160B9B7B061B9BF80
:100DB000380176FD44C07694679400938C001093BC
:100DC0008D00B92DB330E1F0B0FD04C0060D171D44
:100DD000930106C0000F111F0250120922E030E0FB
:100DE000B92DB33068F020938E0030938F000093BC
:100DF00088001093890060928A0070928B003DC039
:100E000000938E0010938F00209388003093890008
:100E100060928A0070928B0071FF10C0B0916D00DB
:100E2000B33060F000918F0010917C001595010F98
:100E300028F022F020928E0000938F001EC066944E
:100E400000938C00B92DB33091F0B0FD03C0060DB6
:100E5000262D03C0000F025022E0B92DB33038F028
:100E600020938E000093880060928A0006C0009351
:100E70008E002093880060928A0000917D0002FD20
:100E80000350013029F495FD0AC0B0E0B7B909C09C
:100E9000023019F4B7E0B7B904C095FDF6CFB6E05B
:100EA000B7B90091A400000F10F4BBE60B27009324
:100EB000A40060FDFECFB2E0B0936E006160B9B7F0
:100EC000B061B9BFB72FB670A1F020917A00309110
:100ED0007B0036952795F8940CB51DB5020F131FAE
:100EE0001BBD0ABD6160B0E1B8BFB9B7B061B9BFA1
:100EF00078940895606120927E0020E067FD20E2F2
:100F000006C0606120927E0020E267FD20E07894B8
:100F100001E076FD11C0B72FB67009F06F7EB09179
:100F20007B00B55048F002E0B55020F003E0B5502A
:100F300008F006E071FD0AE060FD12C0B0917E008D
:100F4000BB2371F071FF08C0B0916D00B33020F089
:100F5000B0916E00BA9519F4789470615CC0AEDF00
:100F6000789400000000F89476FD16C010917B0084
:100F7000173008F017E0B5E01B0F72FD10E183FF9A
:100F8000110F62FF110F71FD12E8B4B56090A1005E
:100F9000B61990F2B10B80F2B0B7B77FB0BFB8B15D
:100FA000B0B7B860B0BFB0917E00B395B0937E008B
:100FB000B8B176FD06C0B1E071FDB2E0BA95F1F7C7
:100FC000B8B1B072B21709F01BC071FF05C003952C
:100FD0000A3008F00395B0CF64FF99CF6F7E3CB51F
:100FE0006DB470907A0080907B00370D681C6BBCEC
:100FF0003ABD6160B0E1B8BFB9B7B061B9BF87CFE2
:10100000B0916D00B23008F482CF64FD80CF0A95B4
:1010100009F092CF7F7E20918E0030918F00F8945E
:10102000B0E1B8BF0CB51DB5020F131F1BBD0ABD43
:10103000E0908800F09089006160B9B7B061B9BFF5
:101040007894B72FB67039F0B0916D0072FFB395F8
:10105000B0936D0009C074FF07C067FD05C064FD53
:1010600003C0BF91BF91DCC4089500E063FF03C0DB
:1010700064FF01C001E0F89410917100B7E01B9F7C
:10108000212D102D7894200F2695179526951795CC
:101090002695179510937100183718F4B8E7B09398
:1010A000710000917100B09172000B1720F0606226
:1010B000C098AC98959860FDFECFE0908A00F090C3
:1010C0008B006160B9B7B061B9BF0895C49AB2E04E
:1010D00095FD07C0F894B0937D00AD98AB9A7894D5
:1010E000EAC0F894B0937D00AD98949A7894E3C0E8
:1010F000C498B3E082FF24C095FD11C002E0F894CB
:10110000B0937D00E6E8F0E00093B30095989498E2
:1011100062FF02C0AC9A01C0AD9A7894CCC002E0E4
:10112000F894B0937D00E6E8F0E00093B300C09837
:10113000AB9862FF02C0AC9A01C0AD9A7894BBC074
:1011400095FD0BC0F894B0937D00E0E7F0E0959832
:1011500062FF01C0AC9A7894AEC0F894B0937D0061
:10116000E0E7F0E0C09862FF01C0AC9A7894A3C0B9
:10117000C49AB4E095FD07C0F894B0937D00AB9895
:10118000949A789498C0F894B0937D009498AB9A10
:10119000789491C0C498B5E082FF24C095FD11C039
:1011A00001E0F894B0937D00ECE7F0E00093B30029
:1011B000AC98AD9862FF02C0C09A01C0AB9A789417
:1011C0007AC004E0F894B0937D00E0E9F0E0009389
:1011D000B300AC98AD9862FF02C0959A01C0949A92
:1011E000789469C095FD0BC0F894B0937D00EAE651
:1011F000F0E0AC9862FF01C0C09A78945CC0F894AB
:10120000B0937D00E6E7F0E0AC9862FF01C0959AEC
:10121000789451C0C49AB6E095FD07C0F894B09395
:101220007D009498AD9A789446C0F894B0937D0070
:10123000AB98AD9A78943FC0C498B1E082FF24C0C7
:1012400095FD11C004E0F894B0937D00E0E9F0E072
:101250000093B300C098AB9862FF02C0959A01C09A
:10126000949A789428C001E0F894B0937D00ECE75C
:10127000F0E00093B3009598949862FF02C0C09A82
:1012800001C0AB9A789417C095FD0BC0F894B09349
:101290007D00E6E7F0E0C09862FF01C0959A78947F
:1012A0000AC0F894B0937D00EAE6F0E0959862FFFA
:1012B00001C0C09A78946F7D089529E630E0F90165
:1012C0002092B300C098AC989598AB98AD9894983C
:1012D0006B7F0895A4EBB0E007E00D9307E00D935A
:1012E00001E00D9304E00D930FEF0D930D9309E0D2
:1012F0000D9302E00D9301E00D9301E00D93A0EC3E
:10130000B0E001E00D9300E00D9304EB0D930FEFBF
:101310000D930D930D9303E00D930FEF0D9301E0EB
:101320000D930FEF0D9305E20D9300ED0D9308E77C
:101330000D9308EC0D9304E00D930FEF0D9301E076
:101340000D9300E00D930AE70D930AE00D9300E082
:101350000D9301E00D9300E00D930FEF0D930895B1
:101360002091BB008B7F233009F48460B091BC00D6
:101370009F7DB1FD90629F7BB091BD00B1FD9064F7
:10138000223011F0886001C0877F08950A95E00F30
:10139000F21DB4910895ECE1F0E00091B400F6DFA5
:1013A000B093D800ECE1F0E00091B500EFDFB0932E
:1013B000D900EAE2F0E00091BA00E8DFB093DA0089
:1013C0000091D300002309F40395013108F001E1F5
:1013D000B02FB00FB00FB093A7001B2FB10FB10FFC
:1013E000B00FB093A800B10FB00FB00FB093A90029
:1013F000B091D0000FEF1CE0B23011F400EA1AE017
:10140000B33011F402E815E00093720010937300FA
:10141000E8E3F0E00091D700B9DFB093A2000895AF
:1014200008952091CA003091CB00B091BC00B33038
:1014300009F43E5097FF02C020E03FEFB32FB21BEC
:101440006B2EB25810F4B2E86B2E00E00395609E4C
:10145000B12DBD57D8F30093AE0008959068E1DF39
:10146000E2D820E030E0B0E16B2ED9D8B0919700FF
:101470002B0F321D6A94C9F7B4E036952795BA95BB
:10148000E1F7822E9F77CDDF0895F894E3E0F0E056
:10149000B9E0B7BFB491B078C1F3F894A895B1B5ED
:1014A000B861B1BDB0E0B1BDB4E0BEBFBFE5BDBF86
:1014B00004DFB0E0B8BBB1E1B7BBB0E0B5BBB8E3A7
:1014C000B4BBB0E0B2BBB0E3B1BB2224A0E0B0E05B
:1014D0002D92AA31E9F7A0E6B0E00FEF2D920A9520
:1014E000E9F7B1E0B093A400F5DECFD2B6B1B460B5
:1014F000B6B90091CC000093AF00B1E0B0936A00A0
:10150000F89495D89FD88FD8A0D88DD8A1D88BD84B
:101510004BD38DD88CD889D8F8940AEF1AEFA0B3A2
:1015200096FDA095A2FF1FC01A95C9F70A95B1F7BD
:10153000E0E0FCE1B591B43E39F4B591B03E21F460
:10154000B591BF3F09F40CC0E0E0F395F395B59178
:10155000B83F49F4B591B43931F4B591BA3A19F4B8
:10156000EE27F6950994FCDE16DF5ADF5ADF00916C
:10157000CC000093AF00A1DEB2E0B3BFB2E0BEBDCD
:10158000B2E0B5BDB1E5B8BFB9BFB0B7B77FB0BFC6
:10159000B8B1B0B7B860B0BF40D8789447DAB3E01C
:1015A00096FDB2E0B5BFB0E4BBBFBB27B064BABF25
:1015B0008D7F3DD8626033E02CE0B0919600BB2374
:1015C00021F42CE03A9509F4A7CF2DD880FFA4CFC1
:1015D0008E7FB0919700B23078F3B92FBF71009130
:1015E000990000939800B0939900B01729F72A95B5
:1015F00021F76D7FB3E096FDB2E0B5BFBB27B064C5
:10160000BABF8D7FB091D600BB2321F48062B92F81
:10161000B0709B2F8F7B2092670007D885FF05C095
:10162000B0916700BA3008F08064F9D702E085FF16
:1016300001C000E0B0919700B017B8F3F89402D859
:1016400001D800D87894F3D720928700E8D7B091DA
:10165000C000B13008F46EC0B0916A00B13008F437
:1016600069C085FD18C0B0919700BF3F08F462C003
:10167000F894F1D77894D9D7B0919700B130C0F7EA
:10168000F894E0D7CED7DED77894CFD7B091970033
:10169000BF3FB0F3BBC2B8E09B2E9068F894C1DEA8
:1016A0007894C3D7F8949F77BCDE80909700B09170
:1016B0009700BF37789408F445C0AFD7F894CBD7DC
:1016C00078949A9451F7CADEB82DB550B093CB00F8
:1016D000AED7F89407D26DD27894BAE09B2E90687A
:1016E000F8949FDE7894A1D7F8949F779ADE809043
:1016F0009700B0919700BF37789478F78ED7F89419
:10170000A1D78FD79FD778949A9449F7A7DEB82DA1
:10171000BB5FB093CA008BD7F894E4D159D27894C8
:1017200084D7F8947EDE7894B0919700BF3F08F498
:1017300098CF6CC200919700B09187000B1710F002
:101740000093870072D701E0B091BC00B35009F458
:1017500005E0B0919700B01708F078CFF8947BD7E8
:101760007AD779D7789463D720926A0020926B0059
:1017700020926C00B0916B00B395B0936B00BF3FAB
:1017800069F5B0916C00B395B0936C00B091CE0048
:1017900009E1BA9559F002E3BA9541F00DE7BA951F
:1017A00029F00AEFBA9511F020926C00B0916C000C
:1017B000B017A0F0B0916C00BA95B0936C00B4EB88
:1017C000B0936B00B091CD00B093AF00F89443D7C5
:1017D0007894B091CC00B093AF0027D722D7B091C6
:1017E0006800BB2319F485FF01C096CE01E085FD9A
:1017F00001C006E0B0919700B01708F4BBCF15D731
:10180000B0916800BB2309F487CEF89456DD20928E
:1018100061002092620020926300522C20926400AA
:101820002092A3007894B091B900BB0FB093A000B0
:1018300020927F00209280002092810020928200DE
:10184000209283002092AC0060E070E02092710052
:10185000B8E0B093AC007860E0D6B2E073FDB1E0E0
:10186000B7B9B6B1B068B064B6B9B6B1B6FDFDCF20
:1018700004B115B1B6B1BF77B6B9112309F00FEFB6
:101880000093AD0036D9B8E0B093AC00786080909A
:10189000BB00B2E0B093BB0063DD8092BB00F89464
:1018A000BFEFB0939C00A0D9B0916100B0939C00B1
:1018B000B0939D00B0939E007894B1E0B093610026
:1018C000B09363005B2EB0936400B093A600B09118
:1018D0009B00B093A500B091BC00B33019F49F7D7C
:1018E00087FD90627160726020926D0093DCA4DCD1
:1018F00094D999D992D997D990D906C0F89430DD66
:1019000078942092AC00777FFCDA1CD7AEDBDEDB6C
:101910008AD9F0DA66FD90D776FF48D876FD76D87A
:10192000A4DBE6DB80D9EDDA66FDA8D79EDB20DC00
:101930007AD9E0DA66FDDCD798DB2CDC74D9E1DA01
:1019400066FD06D892DB66DC6ED9D4DAB2E073FDB0
:10195000B1E0B7B9B6B1B068B064B6B986DB6CDCDB
:1019600062D9C7D871FF20C067FD1EC0B0919F002B
:10197000B0939C00B0939D00B0919B00B093A500E4
:10198000B1E0B093A60018E12CE0B0916D00B11762
:1019900028F07D7F746020936F0006C0B09197009F
:1019A000B13008F0B1CF46C072FF10C067FD0EC065
:1019B000B0916F00BA9511F47B7FA0CFB0936F0008
:1019C000B0919700B13008F09FCF34C020927000E2
:1019D000B0919A00B13058F0B0919F00B0939D0043
:1019E000B0919B00B093A500B1E0B093A600B09178
:1019F0009A000AEFB01708F01DC085FF04C0B0912F
:101A00006800BB23B9F000EF67FF05C0B0919F00ED
:101A1000B0939C0000E2B0917B00B01708F474CF43
:101A2000B0917000B395B0937000B0919700BB2354
:101A300009F002C020927000F8943FDC8090BB0057
:101A4000B2E0B093BB008CDC8092BB0020926100BE
:101A50002092620020926300522C20926400209217
:101A6000A0007E7F7894D9D528DCB6B1B460B6B931
:101A700085FF05C0B0916800BB2309F44DCDB0913E
:101A8000C100B13008F0D1CD71CEEDE0F0E023D04F
:101A9000053A09F01BC0EEE0F0E01DD00A3509F070
:101AA00015C03AE0A4EBB0E0E3E0F0E014D00D9311
:101AB00031963A95D9F738E1A0ECB0E0EFE0F0E0EC
:101AC0000AD00D9331963A95D9F702C003DC0AD0BB
:101AD000E7E2F0E00895E199FECFEEBBFFBBE09AAC
:101AE0000DB308951ED03AE0A4EBB0E0E3E0F0E0DF
:101AF0000D910FD031963A95D9F738E1A0ECB0E0CE
:101B0000EFE0F0E00D9105D031963A95D9F712D07B
:101B10000895E199FECF0DBBEEBBFFBBE29AE19ABF
:101B20000895EDE0F0E00FEFF4DFEEE0F0E00FEF0E
:101B3000F0DF0895EDE0F0E005EAEBDFEEE0F0E045
:101B40000AE5E7DF08953091B0000091B10031302F
:101B500011F40093B400323011F40093B500333027
:101B600011F40093B600343011F40093C8003530FE
:101B700011F40093B700363011F40093BA003730F7
:101B800011F40093C600383011F40093BB003930D3
:101B900011F40093D0003A3011F40093BC003B30B4
:101BA00011F40093BD00089525E041D52A95E9F789
:101BB000089548D54AD54CD54ED533D543D545D5CE
:101BC00047D549D52ED53ED540D542D544D50895E3
:101BD00042D53ED53AD536D524D53DD539D535D59E
:101BE00031D51FD538D534D530D52CD50895809032
:101BF000B0009090B10026D525D524D512D58A9471
:101C0000D1F729D50ED59A94E1F70895F894D1DF4C
:101C10007894CADFC9DFB1E0B093B000B1E0B0930F
:101C2000B1002092B200F894E2DF7894B5E06B2E18
:101C300070909700FCD4B09197007B16C9F7B13033
:101C400018F0BF3F40F107C07EDFF8944BDFB1DFF3
:101C5000B8E0B1BDA9DF6A9459F7B091B200B3956D
:101C6000B093B200B33008F4DECF9EDFB091B10084
:101C7000B395B093B100F894B091B000BA95EEE38B
:101C8000F0E0EB0FF21D049178940395B091B10050
:101C9000B01708F4C6CF88DF87DFB091B000B395E6
:101CA000B093B000B091B000BC3008F4B7CF12DBF5
:0C1CB000F89418DFB8E0B1BD77DFE7CB97
:00000001FF
